:020000040000FA
:42000000FFFF62F73300FFFFFFFFFFFFFFFFFFFFFFFFFFFFFFFFFFFFFFFFFFFFFFFFFFFFFFFFFFFFFFFFFFFFFFFFFFFFFFFFFFFFFFFFFFFFFFFFFFFFFFFFFFFFFFFFFFFFFFFF70
:42004200A00C9481325006CA40190053600A4C81A9325506CA401928034C80613001000000000006988013001324830C900132400618061360022002648001300006C00018FEFE
:420084000015A00254800A50012A800A50012A4005B4800A50012A4005A8002DA00200000000000950012A800E780117E0025C800BD0022A400550012A400248000920013CFE56
:4200C6000004800010000240000800024000080001300002400008000100000000000000000000000000000000000000000000000000000000000000000000000000000010FC48
:42010800000000000000000000000000000000000000000000000000000000000000000000000000000000000000000000000000000000000000000000000000000000003CFE7B
:42014A000001280004800010800220080001200004848000148002500000000000000000000000000000000008080000000000000000000000000000000000000000000080FC71
:42018C0000058000040042400100000000820810011184024000080001000000000000000000000000000000000000000000000000000000000000000000000000000000DCFED0
:4201CE00000000000000000000000000000000000000000000000000000000000000000000000000000013020000000000000000000000000000000000000000000000000CFCD2
:42021000000000000000000000000000000000000000000000000000000000000000000000000000000000000000000000000000000000000000000000000000000000003CFE72
:4202520000000000000000000000000000000000000000000000000000000000000000000000000000C00300000000000000000000000000000000000000000000000000FCFDAE
:42029400000000000000000000000000000000000000000000000000000000000000000000000000004010040000000000000000000000000000000000000000000000002CFFA9
:4202D600000000000000000000000000000000000000000000000000000000000000000000000000000000000000000000000000000000000000000000000000000000003CFEAC
:4203180000000000000000000000000000000000000000000000000000000000000000000000000000C00300000000000000000000000000000000000000000000000000FCFDE7
:42035A00000000000000000000000000000000000000000000000000000000000000000000000000000000000000000000000000000000000000000000000000000000003CFE27
:42039C00000000000000000000000000000000000000000000000000000000000000000000000000000003000000000000000000000000000000000000000000000000003CFDE3
:4203DE00000000000000000000000000000000000000000000000000000000000000000000000000000000000000000000000000000000000000000000000000000000001EFCC3
:42042000000000000000000000000000000000000000000000000000000000000000000000000000000000000000000000000000000000000000000000000000000000003CFE60
:42046200000000000000000000000000000000000000000000000000000000000000000000000000000000000000000000000000000000000000000000000000000000003CFE1E
:4204A4000800000000000000000000000000000000000000000000000000000000000000000000000000000000000000000000000000000000000000000000000000008025FF6A
:4204E6000000000000000000000000000000000000000000000000000000000000000000000000000000000000000000000000000000000000000000000000000000008096FCC2
:42052800000000000000000000000000000000000000000000000000000000000000000000000000000000000000000000000000000000000000000000000000000000003CFE57
:42056A00040000000000000000000000000000000000000000000000000000000000000000000000000000000000000000000000000000000000000000000000000000006DFFDF
:4205AC00000000000000000000000000000000000000000000000000000000000000000000000000000000000000000000000000000000000000000000000000000000003CFED3
:4205EE000000000000000000000000000000000000001018000000000000000000000000000000000000130200000000000000000000000000000000000000000000000014FD7D
:42063000000000000000000000000000000000000000000000000000000000000000000000000000000000000000000000000000000000000000000000000000000000003CFE4E
:4206720000000000000000000000000000000000000000000000000000000000000000000000000000C00300000000000000000000000000000000000000000000000000FCFD8A
:4206B40004000000000000000000000000000000000080000100000000000000000000000000000000401001000000000000000000000000000000000000000000000000A5FF8A
:4206F6000C0000000000000000000000000000000000802800000000000000000000000000000000000000000000000000000000000000000000000000000000000000005CFEB4
:4207380000000000000000000000000000000000000070000000000000000000000000000000000000C00300000000000000000000000000000000000000000000000000B8FE96
:42077A00080000000000000000000000000000000000C0000000000000000000000000000000000000000000000000000000000000000000000000000000000000000080F8FEFF
:4207BC0000000000000000000000000000000000000040800000000000000000000000000000000000000300000000000000000000000000000000000000000000000000F8FD43
:4207FE00000000000000000000000000000000000000100000000000000000000000000000000000000013020000000000000000000000000000000000000000000000002EFF67
:42084000000000000000000000000000000000000000000000000000000000000000000000000000000000000000000000000000000000000000000000000000000000003CFE3C
:4208820000000000000000000000000000000000000000000000000000000000000000000000000000C00300000000000000000000000000000000000000000000000000FCFD78
:4208C400080000000000000000000000000000000000C000010000000000000000000000000000000040080100000000000000000000000000000000000000000000008031FE31
:4209060000000000000000000000000000000000000000420000000000000000000000000000000000000000000000000000000000000000000000000000000000000080F6FEF9
:42094800000000000000000000000000000000000000F0000000000000000000000000000000000000C0030000000000000000000000000000000000000000000000000030FE8C
:42098A00040000000000000000000000000000000000C0400000000000000000000000000000000000000000000000000000000000000000000000000000000000000000E1FF47
:4209CC00000000000000000000000000000000000000C0040000000000000000000000000000000000000300000000000000000000000000000000000000000000000000F4FD31
:420A0E000000000000000000000000000000000000001018020000000000000030210000000000000000000000000000000000000000000000000000000000000000000016FC19
:420A5000000000000000000000000000000000000000000000000000000000000000000000000000000000000000000000000000000000000000000000000000000000003CFE2A
:420A9200000000000000000000000000000000000000000000000000000000003C200000000000000000000000000000000000000000000000000000000000000000000020FCAA
:420AD4000400000000000000000000000000000000008000190800000000000004000000000000000000000000000000000000000000000000000000000000000000008071FF47
:420B16000C000000000000000000000000000000000080228010000000000000000000000000000000000000000000000000000000000000000000000000000000000080D6FF0A
:420B580000000000000000000000000000000000000070001E000000000000003C000000000000000000000000000000000000000000000000000000000000000000000098FEFB
:420B9A00080000000000000000000000000000000000C000180800000000000000000000000000000000000000000000000000000000000000000000000000000000000079FEBA
:420BDC0000000000000000000000000000000000000040149800000000000000300000000000000000000000000000000000000000000000000000000000000000000000CCFFF0
:420C1E00000000000000000000000000000000000000100002000000000000003021000000000000000023010000000000000000000000000000000000000000000000003EFDD2
:420C6000000000000000000000000000000000000000000000000000000000000000000000000000000000000000000000000000000000000000000000000000000000003CFE18
:420CA200000000000000000000000000000000000000000000000000000000003C1000000000000000C00300000000000000000000000000000000000000000000000000D0FC35
:420CE400080000000000000000000000000000000000C0001908000000000000040000000000000000401004000000000000000000000000000000000000000000000080E5FE2A
:420D260000000000000000000000000000000000000000480021000000000000000000000000000000000000000000000000000000000000000000000000000000000080CEFED6
:420D6800000000000000000000000000000000000000F0001E000000000000003C0000000000000000C00300000000000000000000000000000000000000000000000000D0FD6F
:420DAA00040000000000000000000000000000000000C0001808000000000000000000000000000000000000000000000000000000000000000000000000000000000000B9FE6C
:420DEC00000000000000000000000000000000000000C04058000000000000003000000000000000000003000000000000000000000000000000000000000000000000001CFC22
:420E2E0000000000000000000000000000000000000010000A0300080C000000B000000000000000000000000000000000000000000000000000000000000000000000005EFF44
:420E7000000000000000000000000000000000000000000000000000000000000010000000000000000000000000000000000000000000000000000000000000000000002CFF05
:420EB200000000000000000000000000000000000000000008000000000000003C2000000000000000000000000000000000000000000000000000000000000000000000A8FCF6
:420EF400040000000000000000000000000000000000C0001108004020000000040000000000000000000000000000000000000000000000000000000000000000000080B9FD45
:420F36000C0000000000000000000000000000000000000091040040100000000000000000000000000000000000000000000000000000000000000000000000000000800AFD01
:420F7800000000000000000000000000000000000000F0001E000038000000003C0000000000000000000000000000000000000000000000000000000000000000000000A8FD10
:420FBA00080000000000000000000000000000000000C0801808006020000000000000000000000000000000000000000000000000000000000000000000000000000000DDFE32
:420FFC00000000000000000000000000000000000000C00418000020010000003000000000000000000000000000000000000000000000000000000000000000000000006CFD1D
:42103E0000000000000000000000000000000000000050180203000800000000302100000000000000000060240000000000000000000000000000000000000000000000A8FC82
:42108000000000000000000000000000000000000000000000000000000000000000000000000000000000000000000000000000000000000000000000000000000000003CFEF4
:4210C200000000000000000000000000000000000000400000000000000000003C000000000000000000007800000000000000000000000000000000000000000000000080FD7B
:421104000800000000000000000000000000000000008000110800602000000004040000000000000000000822000000000000000000000000000000000000000000000051FD08
:421146000000000000000000000000000000000000008004500400004200000000000000000000000000000000000000000000000000000000000000000000000000000080FFCE
:42118800000000000000000000000000000000000000F0200E000078000000003C000000000000000000007800000000000000000000000000000000000000000000000058FF84
:4211CA00040000000000000000000000000000000000C0401800006000000000000000000000000000000000000000000000000000000000000000000000000000000080C4FD26
:42120C00000000000000000000000000000000000000C0088808006024000000300000000000000000000060000000000000000000000000000000000000000000000000E8FC50
:42124E00000000000000000000000000000000000000000000000000000000000000000000000000000000000000000000000000000000000000000000000000000000001EFC44
:421290002000048000100002400008000120000480001000024000080001200004000000000010000240000800012000048000100002400008000120000480001000020034FCBA
:4212D200000000000000000000000000000000000000000000000000000000000000000000000000000000000000000000000000000000000000000000000000000000003CFEA0
:4213140024000480001000024000080001200004800010000240000800012000040000000000100002400008000120000480001000024000080001200004800010000280EDFDF7
:421356000C00000000000000000000000000000000000000000000000000000020000000000000000000024000000000000000000000000000000000000000000000008032FE37
:4213980020000480001000024000080001200004800010000240000800012000000000000000100002000000000120000480001000024000080001200004800010000200F0FC41
:4213DA0008000000000000000000000000000000000000000000000000000000000000000000000000000000000000000000000000000000000000000000000000000000ADFF1D
:42141C002000048000100002400008000120000480001000024000080001200004000000000010000240000800012000048000100002400008000120000480001000020034FC2C
:42145E00000000000000000000000000000000000000000000000000000000000000000000000000000000000000000000000000000000000000000000000000000000003CFE12
:4214A000000000000000000000000000000000000000000000000000000000000000000000000000000000000000000000000000000000000000000000000000000000003CFED0
:4214E200000000000000000000000000000000000000000000000000000000000000000000000000000000000000000000000000000000000000000000000000000000003CFE8E
:42152400000000000000000000000000000000000000000000000000000000000000000000000000000000000000000000000000000000000000000000000000000000003CFE4B
:42156600000000000000000000000000000000000000000000000000000000000000000000000000000000000000000000000000000000000000000000000000000000003CFE09
:4215A80000000000000000000000000000000000000000000000000000000000000000000000000000000480000000000000000000000000000000000000000000000000F0FE8F
:4215EA00000000000000000000000000000000000000000000000000000000000000000000000000000000000000000000000000000000000000000000000000000000003CFE85
:42162C00000000000000000000000000000000000000000000000000000000000000000000000000000000000000000000000000000000000000000000000000000000003CFE42
:42166E00000000000000000000000000000000000000000000000000000000000000000000000000000000000000000000000000000000000000000000000000000000003CFE00
:4216B00000000000000000000000000000000000000000000000000000000000000000000000000000000000000000000000000000000000000000000000000000000080B4FEC6
:4216F200000000000000000000000000000000000000000000000000000000000000000000000000000000020000000000000000000000000000000000000000000000003EFC7A
:4217340000000000000000000000000000000000000000000000000000000000000000000000000000000000000000000000000000000000000000000000000000000080B4FE41
:421776000000000000000000000000000000000000000000000000000000000000000000000000000000810000000000000000000000000000000000000000000000000034FF7D
:4217B800000000000000000000000000000000000000000000000000000000000000000000000000100000000000000000000000000000000000000000000000000000003CFFA4
:4217FA000000000000000000000000008001000000140000000000000000000000000000000000000280000100000000000000000000000000000000000000000000000040FE57
:42183C00000000000000000000000000000020000012410000000240000000000000000000000000088000000000000000000000000000000000000000000000000000007CFDB4
:42187E000000000000000000000000000000000000048400000000000000000000000000000000000200000000000000000000000000000000000000000000000000000090FE10
:4218C0000000000000000000000000000000000100000000000002400000000000000000000000000000000000000000000000000000000000000000000000000000000008FC9F
:421902000000000000000000000000000000000000000000200000A00000000000000000000000000000000000000000000000000000000000000000000000000000000034FEB1
:42194400080000000000000000000000000000000000008000000000000000000004000000000000000040000000000000000000000000000000000000000000000000007CFE1B
:42198600000000000000000000000000000000000000000000000000000000000000000000000000000000000000000000000000000000000000000000000000000000003CFEE5
:4219C80000000000000000000000000000000000000000000000000000000000880000000000000000000000000000000000000000000000000000000000000000000040D2FC47
:421A0A00000000000000000000000000000000000000000000000000000000000000000000000000000000000000000000000000000000000000000000000000000000003CFE60
:421A4C00000000000000000000000000000000000000000000000000000000000000000000000000000002000000000000000000000000000000000000000000000000003CFC1E
:421A8E00000000000000000000000000000000000000000000000000000000000000000000000000000000000000000000000000000000000000000000000000000000003CFEDC
:421AD000000000000000000000000000000000000000000000000000000000000000000000000000000000000000000000000000000000000000000000000000000000003CFE9A
:421B12000000000000000000000000000000000000000000000000000000000004000000000000000000000000000000000000000000000000000000000000000000000038FE57
:421B540000000000000000000000000000000000000000000000000008000000000000000000000000000000000000000000000000000000000000000000000000000000BCFE8D
:421B9600000000000000000000000000000000000000000004000040000000000000000000000000000000000000000000000000000000000000000000000000000000007CFE4F
:421BD800000000000000000000000000000000000000100000000000000000000000000000000000000000000000000000000000000000000000000000000000000000003CFF80
:421C1A0000000000000000000000000000000000000010400A000008000000000000000000000000000000000000000000000000000000000000000000000000000000005EFFC9
:421C5C00000000000000000000000000000000000000400024000000000000000000000000000000000000000000000000000000000000000000000000000000000000001CFCCA
:421C9E00000000000000000000000000000000000000000100000000000000000000000000000000000000000000000000000000000000000000000000000000000000002CFFD8
:421CE000000000000000000000000000000000000000200000100000000000000000000000000000000000000000000000000000000000000000000000000000000000003CFD59
:421D2200000000000000000000000000000000000000000000000000000000000000000000000000000000000000000000000000000000000000000000000000000000003CFE45
:421D6400000000000000000000000000000000000000000000000000000000000000000000000000000000000000000000000000000000000000000000000000000000003CFE03
:421DA6000A0000000000000000004000000100200400800000000000000000000000000000000000000000000000000000000000000000000000000000000000000000C08CFDC3
:421DE80000000000000000000000000000000100000000000000000000000000000800000000000000020000000000000000000000000000000000000000000000000040E3FE8D
:421E2A000003000000800100030010000024000810A0200050000A400100800000200000000000000010000010000000000000000000000000000000000000000000000098FFF1
:421E6C0000000000000000000000000000000000002010000000082000048004200400000000000010800640020000000000000000000000000000000000000000000000BCFE9E
:421EAE000000000000000000000000000000000000000000000000100002400000000000000000000000000000000000000000000000000000000000000000000000000008FD9B
:421EF0000000000000000000000000000000000000000000000000000000000010080000000000000480001000000000000000000000000000000000000000000000000064FFA1
:421F32000000000000000000000000000000000000004000000000000000000000000000000000000000000000000000000000000000000000000000000000000000000078FEB7
:421F7400000000000000000000000000000000000000000000000000000000000000000000000000000000000000000000000000000000000000000000000000000000003CFEF1
:421FB600000000000000000000000000000000000000200200000000000000000000000000000000000000000000000000000000000000000000000000000000000000001CFEAD
:421FF800000000000000000000000000000000000000000000000000000000000000000000000000000000000000000000000000000000000000000000000000000000003CFE6D
:42203A00020000000000000000000000000000000000000000000000000000000000000000000000000000000000000000000000000000000000000000000000000000406BFDBA
:42207C00000000000000000000000000000000000000000000000000000000000000000000000000000000000000000000000000000000000000000000000000000000002DFFF6
:4220BE000000000000000000000000000000000000000000000000000000000000000000000000000000000000000000000000000000000000000000000000000000004078FE2A
:42210000000000000000000000000000000000000000000000000000000000002000000000000000008000100000000000000000000000000000000000000000000000009CFF52
:4221420000000000000000000000000000000000000000800000000000000000000000000000000000000000000000000000000000000000000000000000000000000000BCFE21
:42218400000000000000000000000000000000000000000000020000000000000000000000000000000000000000000000000000000000000000000000000000000000001CFEFD
:4221C600000000000000000000000000000000000000000000000000000000000000000000000000000000000000000000000000000000000000000000000000000000003CFE9D
:42220800000000000000000000000000000000000000000000000000000000000000000000000000000000000000000000000000000000000000000000000000000000003CFE5A
:42224A0000000000000000000000000000000000000000005808030100000000000000000000C00001000000000C0400040000000000000000000000000000000000000008FD14
:42228C00000000000000000000000000000000000000000000000000000000000000000000000000000000000000000000000000000000000000000000000000000000003CFED6
:4222CE0000000000000000000000000000000000000000001ED0030200000000000000000000F08000000000000F0800302000000000000000000000000000000000000098FF6D
:422310000000000000000000000000000000000000000000024020000000000000000000000010040000000000410000000200000000000000000000000000000000000028FDAD
:42235200000000000000000000000000000000000000000000000000000000000000000000000000000000000000000000010000000000000000000000000000000000002CFE1E
:4223940000000000000000000000000000000000000000001EC0030000000000000000000000F00000000000000F00000C20000000000000000000000000000000000000ECFF10
:4223D600000000000000000000000000000000000000000000000000000000000000000000000000000000000000000000200000000000000000000000000000000000003CFC6D
:4224180000000000000000000000000000000000000000001800030000000000000000000000C00000000000000C0000000000000000000000000000000000000000000098FC07
:42245A0000000000000000000000000000000000000000005800030000000000000000000000C00003110000000C04000000000000000000000000000000000000000000CEFF34
:42249C0000000000000000000000000000000000000000000008000200000000000000000000000000000000000000000000000000000000000000000000000000000000BCFC3C
:4224DE0000000000000000000000000000000000000000001EC8030100000000000000000000F08000000000000F00000000000000000000000000000000000000000000A8FCAF
:42252000080000000000000000000000000000000000000002410000000000000000000000001008800800000041100000000000000000000000000000000000000000806DFD53
:4225620000000000000000000000000000000000000000000000000000000000000000000000000050040000000000000000000000000000000000000000000000000080D6FD90
:4225A40000000000000000000000000000000000000000001EC0030000000000000000000000F00006000000000F0000000000000000000000000000000000000000000040FDD2
:4225E600040000000000000000000000000000000000000000000000000000000000000000000000000000000000000000000000000000000000000000000000000000006DFF43
:4226280000000000000000000000000000000000000000001800030000000000000000000000C00080020000000C0000000000000000000000000000000000000000000030FED9
:42266A0000000000000000000000000000000000000000005808030100000000000000000000C048020000000041000004000000000000000000000000000000000000003CFC43
:4226AC00000000000000000000000000000000000000000000000000000000000000000000000000000000000000020000000000000000000000000000000000000000001CFED0
:4226EE0000000000000000000000000000000000000000001EC8030100000000000000000000F08018000000000002000020000000000000000000000000000000000000C4FC56
:422730000400000000000000000000000000000000000000024108000000000000000000000010040004000000400000000200000000000000000000000000000000000045FD7C
:422772000C000000000000000000000000000000000000000000000000000000000000000000000040080000004000000001000000000000000000000000000000000000A4FEEE
:4227B40000000000000000000000000000000000000000001EC0030000000000000000000000F00006000000000304003C2000000000000000000000000000000000000030FC7D
:4227F6000800000000000000000000000000000000000000000000000000000000000000000000000000000000000000002000000000000000000000000000000000008034FCC9
:4228380000000000000000000000000000000000000000001800030000000000000000000000C00080200000002404000000000000000000000000000000000000000000D8FEE5
:42287A0000000000000000000000000000000000000000001808030000000000000000000000000002000000002C04000400000000000000000000000000000000000000DCFEE9
:4228BC00000000000000000000000000000000000000000000000002000000000000000000000000000000000000000000000000000000000000000000000000000000003CFCA0
:4228FE0000000000000000000000000000000000000000001EC8030100000000000000000000000000000000000F0000002000000000000000000000000000000000000050FE31
:422940000400000000000000000000000000000000000000024108000000000000000000000000000004000000411000000200000000000000000000000000000000000011FDA1
:422982000C000000000000000000000000000000000000000000000000000000000000000000000040080000000000000001000000000000000000000000000000000000A0FE20
:4229C40000000000000000000000000000000000000000001EC0030000000000000000000000000006000000000F00000C200000000000000000000000000000000000007CFF34
:422A06000800000000000000000000000000000000000000000000000000000000000000000000000000000000000000002000000000000000000000000000000000008034FCB6
:422A480000000000000000000000000000000000000000001800030000000000000000000000000098200000000C0000300000000000000000000000000000000000000040FEFF
:422A8A00000000000000000000000000002010010000000018080B600100000000000000000000001A00000000410000B000000000000000000000000000000000000000B6FE8E
:422ACC00000000000000000000000000000000000000000000000001200000000000000000000000000000000000020000080000000000000000000000000000000000009CFD04
:422B0E0000000000000000000000000000000000000000001ED0037A20000000000000000000000000000000000002003C000000000000000000000000000000000000007CFF41
:422B5000040000000000000000000000000011010000000002402008000000000000000000000000000400000040000004040000000000000000000000000000000000800DFDED
:422B92000C0000000000000000000000000051000000000000000000000000000000000000000000400800000040000000000000000000000000000000000000000000800AFC96
:422BD40000000000000000000000000000E00000000000001EC0037800000000000000000000000006000000000304003C000000000000000000000000000000000000009CFDA4
:422C1600080000000000000000000000008001000000000000000000000000000000000000000000000000000000000000000000000000000000000000000000000000002DFEC8
:422C58000000000000000000000000000080800000000000180003600000000000000000000000008020000000240400300000000000000000000000000000000000000084FF44
:422C9A0000000080000000000000000000200000000000000200030000000000000000000000000082000000002C04003400000000000000000000000000000000000000D4FE9B
:422CDC0000000000000000000000000000000000000000000000000200000000000000000000000008100000000000000000000000000000000000000000000000000000ACFCF4
:422D1E00000000000002000000000000000000000000000000C0030000000000000000000000000000000000000F080000200000000000000000000000000000000000008CFEED
:422D60000400000016000000000000000080110100000000406040000000000000000000000000004020000000810000000200000000000000000000000000000000000095FE2F
:422DA2000C00000040020000000000000000840000000000000000000000000000000000000000008000000000000000000100000000000000000000000000000000000068FC38
:422DE40000000080070000000000000000E001000000000006C4030000000000000000000000000006080000000F00000C20000000000000000000000000000000000000F0FC43
:422E26000800000006000000000000000080010000000000180000000000000000000000000000000000000000000000002000000000000000000000000000000000008008FE1D
:422E680000000000060200000000000000808500000000004004030000000000000000000000000000080000000C0000000000000000000000000000000000000000000064FC60
:422EAA00000000800000000000000000002000000000104218480000000000000000000000000000820800000041000030010000000000000000000000000000000000000EFC8E
:422EEC0000000000000000000000000000000000000000000000030000000000000000000000000000000000000002000008000000000000000000000000000000000000ACFDEE
:422F2E0000000000060200000000000000000000000000801E00800000000000000000000000000000000000000002003C0000000000000000000000000000000000000018FEE7
:422F70000400000010000000000000000080110100000004020808000000000000000000000000008008000000400000040400000000000000000000000000000000008079FD9D
:422FB2000C00000026000000000000000000080100000004000020000000000000000000000000005004000000400000000000000000000000000000000000000000008088FDE5
:422FF40000000080010400000000000000E00100000030401EC0800000000000000000000000000006000000000304003C000000000000000000000000000000000000000CFE14
:423036000800000006000000000000000080010000000000000000000000000000000000000000000000000000000000000000000000000000000000000000000000008081FCCC
:4230780000000000160400000000000000801102000040421800A000000000000000000000000000800200000024040030000000000000000000000000000000000000005CFCFD
:4230BA0000000080000000000000000000A01001000010428220036101000000000000000000000002000000002C2400B000000000000000000000000000000000000000CCFF7D
:4230FC0000000000000000000000000000000000000000000000000020000000000000000000000000000000000000000008000000000000000000000000000000000000BCFCB2
:42313E00000000000604000000000000008000000000008000D0037800000000000000000000000000000000000F08003C10000000000000000000000000000000000000ACFCEF
:4231800008000000000000000000000000001101000000048040400808000000000000000000000000040000004100008400000000000000000000000000000000000000E1FE37
:4231C20000000000160100000000000000004500000000044004000000000000000000000000000040080000000080210000000000000000000000000000000000000000FCFD45
:4232040000000080010000000000000000E001000000304006C003780000000000000000000000001E000000000FE0013C000000000000000000000000000000000000000CFD22
:423246000400000006010000000000000080810000000000000000000000000000000000000000000000000000000000000000000000000000000000000000000000008058FC66
:4232880000000000060000000000000000800100000040420820036000000000000000000000000080200000000C0004310000000000000000000000000000000000000070FE21
:4232CA00000000000000000000000000000000000000000000000000000000000000000000000000000000000000000000000000000000000000000000000000000000003CFE88
:42330C002000048000100002400008000120000480001000024000080001200004000000000010000240000800012000048000100002400008000120000480001000020034FC1D
:42334E00000000000000000000000000000000000000000000000000000000000000000000000000000000000000000000000000000000000000000000000000000000003CFE03
:4233900024000480001000024000080001200004800010000240000800012000040000000000100002400008000120000480001000024000080001200004800010000280EDFD5B
:4233D2000C00000000000000000000000000000000000000100002400000000000000000000080000000000000080000200000000000000000000000000000000000008068FFCC
:4234140020000480001000024000080001200004800010000000000000012000040000000000000002400008000020000080001000024000080001200004800010000200ACFFF8
:423456000800000000000000000000000000000000000000000000000000000000000000000000000000000000000000000000000000000000000000000000000000008025FF88
:423498002000048000100002400008000120000480001000024000080001200004000000000010000240000800012000048000100002400008000120000480001000020034FC90
:4234DA00000000000000000000000000000000000000000000000000000000000000000000000000002000000000000010000000000000000000000000000000000000000CFF75
:42351C00000000000000000000000000000000000000000000000000000000000000000000000000000000000000000000000000000000000000000000000000000000003CFE33
:42355E00000000000000000000000000000000000000000000000100000000000000000000000000000000000000000000000000000000000000000000000000000000002CFFFF
:4235A000000000000000000000000000000000000000000000000000000000000000000000000000000000000000000000000000000000000000000000000000000000003CFEAF
:4235E200000000000000000000000000000000000000000000000000000000000000000000000000000000000000000000000000000000000000000000000000000000003CFE6D
:42362400000000000000000000000000000000000000000000004000000000000000000000000010000000000000010000000000000000000000000000000000000000005EFDB8
:4236660000000000000000000000000000000000000000000800000000000000000000000000000000000000000400000400000000000000000000000000000000000000B4FE60
:4236A800000000000000000000000000000000000000000000000001000000000000000000000000000000000000000000000000000000000000000000000000000000003CFFA4
:4236EA000000000000000000000000000000000000000000000000000000000000000000000000800000000000000000000000000000000000000000000000000000004070FE70
:42372C00000000000000000000000000000000000000000000000000000000000000000000000000200000000000000000000000000000000000000000000000000000003CFC03
:42376E000A0000000000000000000000000000000000000000000000000000000000000000000000000000000000080000000000000000000000000000000000000000001CFEED
:4237B000000000000000000000000000000000000000000000000000000000000000000000000000000000000000000000000000000000000000000000000000000000003CFE9D
:4237F20000000000000000000000000000000000000000000000000000000000000000000000000008040200000000000000000000000000000000000000000000000000B8FCD3
:423834000000000000000000000000000004000000000000000000000000000000000000000000000000000000000000000000000000000000000000000000000000000038FE18
:423876000000000000000000000000000008000000000000500051000000000000000000000000005488000000040040A00500000000000000000000000000000000000090FD15
:4238B800000020000400000000000000000040000402410050100940000000000000000000008001A21101000008400A080000000000000000000000000000000000000000FEED
:4238FA000000000000000000000000000000000100048400000002000000000000000000000000000000020000000000000000000000000000000000000000000000000080FE81
:42393C000000200004000000000000000000000020000000100000400000000000000000000040000000000000040000000000000000000000000000000000000000000028FD4C
:42397E000000000002000000000000000000400000000000000000000000000000000000000000002800000000000000000800000000000000000000000000000000000018FE7F
:4239C00008000000000000000000000000000000000000000000000000000000000000000000000000000000000000000000000000000000000000000000000000000000BCFE03
:423A0200000000000000000000000000000000000000000020000000000000000000000000000000000000000000000000000000000000000000000000000000000000001CFC4A
:423A44000000000000000000000000000000000000000000488000100000000000000000000000000000000000000000000000000000000000000000000000000000000028FF41
:423A8600000000000000000000000000000000000000000000000000000000000000000000000002000000000020000000000000000000000000000000000000000000001CFEC2
:423AC800000000000000000000000000000000000000000000000000000000000000000000000000000000000000000000000000000000000000000000000000000000003CFE82
:423B0A000000000000000000000000000000000000004000000000000000000000000000000000000000000000000000000000000000000000000000000000000000000078FEC3
:423B4C00000000000000000000000000000000000000000000200000000000000000000000000000020000000000000000000000000000000000000000000000000000001CFCFD
:423B8E0000000000000000000000000000000000000000000040000800000000000000000000000000000000000000000000000000000000000000000000000000000000F0FEBF
:423BD000000000000000000000000000000020000000000000000000000000000000000000000000000000000000000000040000000000000000000000000000000000005CFC37
:423C120000000000000000000000000000000000000000000480000000000000000000000000000010000000000200000000000000000000000000000000000000000000F0FDED
:423C5400000000000100000000000000000000000000000000000000000000000000000000000000000000000000200000000000000000000000000000000000000000002CFDE4
:423C96000000000000000000000000000000020000000000000000000000000000000000000000000004000000000000000000000000000000000000000000000000000038FCB2
:423CD800000000000000000000000000004000000000000000000000000000000000000000000000000000000000000000000000000000000000000000000000000000007CFEF0
:423D1A0000000000080000000000000000800000000000000000000000000000000000000000000000000000000000000000000000000000000000000000000000000000B4FE2D
:423D5C00000000000000000000000000000000000000000000000000000000000000000000000000000000000000000000000000000000000000000000000000000000003CFEEB
:423D9E00000000000001000000000000000000000000000000000000000000000000000000000000000000000000000000000000000000000000000000000000000000003CFFA7
:423DE00000000000000000000000000000000000000000000000000000000000000000000000000008000000000000000000000000000000000000000000000000000000BCFEDF
:423E220004000000000000000000000000000000200010000000000000000000000000000000000008000000000000000000000000000000000000000000000000000040BAFD2B
:423E6400400000000020000008000000000000001000000000000100000000000000000000000000000400000000804010000000000000000000000000000000000000000CFCC7
:423EA60020000000001000001000000000000000301420000044500000000000000000000000000084120000000020000500000000000000000000000000000000000000B0FE39
:423EE80000000080000000000201000000400048001090001882210A001200000000000000000000100000000019409E08100D0000000000000000000000000000000000F4FFF7
:423F2A0000000000000000008000000000000000000000000480000000000000000000000000000000000000000000000000000000000000000000000000000000000000F8FE5B
:423F6C0000000000000000000800000000000000000040000804000000000000000000000000000008000000000400000000010000000000000000000000000000000000ECFFC7
:423FAE000000000000000000000000000000000000000002400000000000000000000000000000000010000000000000000000000000000000000000000000000000000008FC7B
:423FF0000000000010010000000000000000040000008000001000000000000000000000000000000000000000080040800000000000000000000000000000000000000020FE04
:42403200100000000000000000000000000000000000000000000000000000000000000000000000000000000000000000000000000000000000000000000000000000001EFD21
:42407400000000000000000000000000000000020000000000000000000000000000000000000000000000000000000000000000000000000000000000000000000000001CFEEE
:4240B600100000000000000000000000000000000000800000200000000000000000000000000000000000000008000000000000000000000000000000000000000000003CFDD7
:4240F800000000000000000000000000000000000000000000000000000000000000000000000000000000000000000000000000000000000000000000000000000000003CFE4C
:42413A00000000000000000000000000000000000000000000000000000000000000000000000000000000000000000000000000000000000000000000000000000000003CFE09
:42417C000000000000000000000000000000000000000000100002400000000000000000000020000000000000000000000000000000000000000000000000000000000028FD6A
:4241BE000000000000000000000000000000000000000000000000000000000000000000000000000000000000000000000000000000000000000000000000000000004078FE09
:42420000000000000000000000000000000001000000000000000000000000000000000000000000000000000000000000000000000000000000000000000000000000003CFF40
:42424200000000000000000000000000000000000000000000000000000000000000000000000000000000000000000000000000000000000000000000000000000000002DFF0E
:424284000000000000000000000000000000000000000000000000000000000000000000000000004000000000000000000000000000000000000000000000000000000078FE42
:4242C60000000000000000000023620C0C040030010000000000000000000000000000000000000000000000000000000000000000980000000000000000000000000000CCFC84
:42430800000000000000000000000000000000002000000000000000000000000000000000000000000000000000000000000000000010000000000000000000000000000CFF38
:42434A000000000000000000C00379000F00003C0000000000000000000000000000000000000000000000000000000000000000001E000000000000000000000000000064FE2A
:42438C0000000000000000004010088141080004400000000000000000000000000000000000000000000000000000000000000000821000000000000000000000000000D4FD26
:4243CE00000000000000000000000000000000000000000000000000000000000000000000000000000000000000000000000000000000000000000000000000000000003CFE73
:424410000000000000000000C00378000F00003C0000000000000000000000000000000000000000000000000000000000000000001E000000000000000000000000000074FF53
:42445200000000000000000000000000000000000000000000000000000000000000000000000000000000000000000000000000000000000000000000000000000000003CFEEE
:424494000000000000000000000360000C000030000000000000000000000000000000000000000000000000000000000000000000180000000000000000000000000000B4FD7E
:4244D600000000000000000240000000000000000000000000000000000000000000000000000000000000000000000000000000000000000000000000000000000000003AFE2A
:42451800000000000000000000000000000000000000000000000000000000000000000000000000000000000000000000000000000000000000000000000000000000003CFE27
:42455A000000000000000018000001000000000000000000000000000000000000000000000000000000000000000000000000000000000000000000000000000000000034FFD3
:42459C000800000000000000110B00000000000000000000000000000000000000000000000000000000000000000000000000000000000000000000000000000000008085FFB5
:4245DE00000000000000009804400000000000000000000000000000000000000000000000000000000000000000000000000000000000000000000000000000000000802CFE15
:424620000000000000000006C00300000000000000000000000000000000000000000000000000000000000000000000000000000000000000000000000000000000000024FC6F
:424662000400000000000018040300000000000000000000000000000000000000000000000000000000000000000000000000000000000000000000000000000000000023FDD3
:4246A4000000000000000058000B020000000000000000000000000000000000000000000000000000000000000000000000000000000000000000000000000000000000F4FC7F
:4246E6000000000000000000400008000000003020000000000000000000000000000000000000000000000000000000000000000018030000000000000000000000000008FED9
:42472800000000000000000000000000000000000000000000000000000000000000000000000000000000000000000000000000000000000000000000000000000000003CFE15
:42476A000000000000000000000301200000003C0000000000000000000000000000000000000000000000000000000000000000001E0000000000000000000000000000C0FCD3
:4247AC000400000000000000000860010000000404000000000000000000000000000000000000000000000000000000000000000082100000000000000000000000000079FD4E
:4247EE000C000000000000000013000000000000000000000000000000000000000000000000000000000000000000000000000000000000000000000000000000000000CCFF9F
:424830000000000000000000C00079400000003C0000000000000000000000000000000000000000000000000000000000000000001E0000000000000000000000000000A0FED5
:424872000800000000000000000360000000000000000000000000000000000000000000000000000000000000000000000000000000000000000000000000000000008064FEB7
:4248B40000000000000000000093600A0000003000000000000000000000000000000000000000000000000000000000000000000018000000000000000000000000000074FE0B
:4248F600000000000000001811230A00000000000000000000000000000000000000000000000000000000000000000000000000000000000000000000000000000000002CFE00
:42493800000000000000000000000000000000000000000000000000000000000000000000000000000000000000000000000000000000000000000000000000000000003CFE03
:42497A00000000000000001EC0036000000000000000000000000000000000000000000000000000000000000000000000000000000000000000000000000000000000005CFC62
:4249BC00040000000000000261000444000000000000000000000000000000000000000000000000000000000000000000000000000000000000000000000000000000002DFEDF
:4249FE000C0000000000000000006010000000000000000000000000000000000000000000000000000000000000000000000000000000000000000000000000000000008CFF70
:424A4000000000000000001EC00318000000000000000000000000000000000000000000000000000000000000000000000000000000000000000000000000000000000024FC1B
:424A82000800000000000000000060100000000000000000000000000000000000000000000000000000000000000000000000000000000000000000000000000000008044FFB7
:424AC4000000000000000018000360010000000000000000000000000000000000000000000000000000000000000000000000000000000000000000000000000000000074FFC1
:424B0600000000000000000240006001000000000000000000000000000000000000000000000000000000000000000000000000000000000000000000000000000000005AFF71
:424B4800000000000000000000000020000000000000000000000000000000000000000000000000000000000000000000000000000000000000000000000000000000001CFCF3
:424B8A0000000000000000000803780000000000000000000000000000000000000000000000000000000000000000000000000000000000000000000000000000000000FCFE6C
:424BCC00040000000000005800A008810000000000000000000000000000000000000000000000000000000000000000000000000000000000000000000000000000008035FC71
:424C0E000C00000000000000012300000000000000000000000000000000000000000000000000000000000000000000000000000000000000000000000000000000008044FD73
:424C5000000000000000001ED00379000000000000000000000000000000000000000000000000000000000000000000000000000000000000000000000000000000000044FC78
:424C92000800000000000018100001000000000000000000000000000000000000000000000000000000000000000000000000000000000000000000000000000000000097FD1B
:424CD4000000000000000058000B600000000000000000000000000000000000000000000000000000000000000000000000000000000000000000000000000000000000B4FE29
:424D16000000000000000002400008000000003020000000000000000000000000000000000000000000000000000000000000000000000000000000000000000000000030FF92
:424D5800000000000000000000000000000000000000000000000000000000000000000000000000000000000000000000000000000000000000000000000000000000003CFEDF
:424D9A000000000000000018080060100000003C1000000000000000000000000000000000000000000000000000000000000000000000000000000000000000000000000CFCF3
:424DDC000400000000000040000000040000000401000000000000000000000000000000000000000000000000000000000000000000000000000000000000000000000039FE11
:424E1E000C00000000000018028360240000000000000000000000000000000000000000000000000000000000000000000000000000000000000000000000000000000058FECF
:424E60000000000000000006C00378000000003C0000000000000000000000000000000000000000000000000000000000000000000000000000000000000000000000009CFFF8
:424EA200080000000000001800030020000000000000000000000000000000000000000000000000000000000000000000000000000000000000000000000000000000803CFCD3
:424EE4000000000000000018050360010000003000000000000000000000000000000000000000000000000000000000000000000000000000000000000000000000000030FDAE
:424F2600000000000000000240000800000000000000000000000000000000000000000000000000000000000000000000000000001803130000000000000000000000001AFCBB
:424F6800000000000000000000000000000000000000000000000000000000000000000000000000000000000000000000000000000000000200000000000000000000001CFCED
:424FAA00000000000000000000036000000000000000000000000000000000000000000000000000000000000000000000000000001EC803010000000000000000000000F4FD87
:424FEC0004000000000000000020024400000000000000000000000000000000000000000000000000000000000000000000000000424010000000000000000000000080E1FC2A
:42502E000C00000000000018042360010000000000000000000000000000000000000000000000000000000000000000000000000000000000000000000000000000008078FD9F
:42507000000000000000001EC0801810000000000000000000000000000000000000000000000000000000000000000000000000001EC0030000000000000000000000008CFF0C
:4250B20008000000000000180003604000000000000000000000000000000000000000000000000000000000000000000000000000000000000000000000000000000000C3FD39
:4250F4000000000000000018008B60000000000000000000000000000000000000000000000000000000000000000000000000000018000300000000000000000000000054FE0A
:425136000000000000000002400008000C04003020000000000000000000000000000000000000000000000000000000000000000098006300004C100030060000000000A8FC5C
:42517800000000000000000000000000000000000000000000000000000000000000000000000000000000000000000000000000000010000000000000000000000000002CFFBA
:4251BA000000000000000000000000200F04003C0000000000000000000000000000000000000000000000000000000000000000001EC80301000F00003C00000000000080FF90
:4251FC000400000000000000000060012100000440000000000000000000000000000000000000000000000000000000000000000042401000000101000440000000000079FE58
:42523E000C00000000000058000B00020000000000000000000000000000000000000000000000000000000000000000000000000000000000000000000000000000000014FCAD
:42528000000000000000001EC80379200F00003C0000000000000000000000000000000000000000000000000000000000000000001EC00300000F00003C000000000000FCFDFA
:4252C2000800000000000000000060000000000000000000000000000000000000000000000000000000000000000000000000000000000000000000000000000000008054FE70
:425304000000000000000000059060200C00003000000000000000000000000000000000000000000000000000000000000000000018000300000C00003000000000000098FC2B
:42534600000000000000000000000000000000000000000000000000000000000000000000000000000000000000000000000000000000000000000000000000000000001EFC0B
:425388002000048000100002400008000120000480001000024000080001200004000000000010000240000800012000048000100002400008000120000480001000020034FC81
:4253CA00000000000000000000000000000000000000000000000000000000000000000000000000000000000000000000000000000000000000000000000000000000003CFE67
:42540C0024000480001000024000080001200004800010000240000800012000040000000000100002400008000120000480001000024000080001200004800010000280EDFDBE
:42544E000C00000000000010000240000800002000000000000000000000000000000000000000000000000000000000000000000010000200000800002000000000008034FEAA
:42549000200004800010000000000000002000008000100002400008000120000400000000001000024000080001200004800010000000000800002000008000100002003CFC06
:4254D200080000000000000000000000000000000000000000000000000000000000000000000000000000000000000000000000000000000000000000000000000000008FFD04
:425514002000048000100002400008000120000480001000024000080001200004000000000010000240000800012000048000100002400008000120000480001000020034FCF3
:42555600000000000000000000000000000000000000000000000000000000000000000000000000000000000000000000000000000000000000000000000000000000003CFED9
:42559800000000000000000000000000000000000000000000000000000000000000000000000000000000000000000000000000000000000000000000000000000000003CFE97
:4255DA00000000000000000000000000000000000000000000000000000000000000000000000000000000000000000000000000000000000000000000000000000000003CFE55
:42561C00000000000000000000000000000000000000000000000000000000000000000000000000000000000000000000000000000000000000000000000000000000003CFE12
:42565E00000000000000000000000000000000000000000000000000000000000000000000000000000000000000000000000000000000000000000000000000000000003CFED0
:4256A00000000000000000020000020000040000200000000000000000000000000000000000000000000000000000000000000000000800000000000000200000000000B0FECA
:4256E200000000000000000000000000000000000000000000000000000000000000000000000000000000000000000000000000000000000000000000000000000000003CFE4C
:42572400000000000000000000000000000000000000000000000000000000000000000000000000000000000000000000000000000000000000000000000000000000001EFC29
:425766000000000000000000000000000000000000000000000000000000000000000000000000000000000000000000000000000002400000000000000400000000000058FC67
:4257A800000000000000000000000000000000000000000000000000000000000000000000000000000000000000000000000000000000000000001000000000000000002CFE85
:4257EA0000000000000000008000000000000008000000000000000000000000000000000000000000000000000000000000000000008000000000000000000000000000BCFEBB
:42582C00000000000000000000000000000000000000000000000000000000000000000000000000000000000000000000000000000000000000000000000000000000003CFE00
:42586E00000000000000000000000000000000000000000000000000000000000000000000000000000000000000000020000000000000000000000000000000000000001CFCC0
:4258B0000000000000000000000000000004000008000000000000000000000000000000000000000000000000000000000400000000000000000000000000000000000070FE38
:4258F20000000000000000000000000A00880000200000000000000000000000000000000000000000000000000000000820008002000400000000000000000000000000F8FE1E
:4259340000000000008000100802100A18010400000000000000000000000000000000000000000000000000000000002000000002000000000000000000000000000000C0FE80
:42597600000000000000000000000000000000000000000000000000000000000000000000000000000000000000000000000000000000000000000000000000000000003CFEB5
:4259B8000000000000800010000200400408000000000000000000000000000000000000000000000000000000000000200000000000000000000000000000000000000068FC4B
:4259FA000800000000000008000120000000000000000000000000000000000000000000000000000000000000000000000000000000000000000000000000000000000095FFA6
:425A3C0000000000000000400008400000000000000000000000000000000000000000000000000000000000000000000000000000000000000000000000000000000040E9FF78
:425A7E00000000000000000000000000000000000000000000000000000000000000000000000000000000000000000000000000000000000000000000000000000000003CFEAC
:425AC000000000000000000000000000000000000000000000000000000000000000000000000000000000000000000000000000000000000000000000000000000000003CFE6A
:425B02000000000000000000000200800000000400000000000000000000000000000000000000000000000000000000000000000000000000000100000000000000004000FE9C
:425B4400000000000000000000000000000000000000000000000000000000000000000000000000000000000000000000000000000000000000000000000000000000003CFEE5
:425B860000000000000000000000080004000000080000000000000000000000000000000000000000000000000000000000000000080480000000000000000000000000B8FE87
:425BC800000000000000000020000000000000000000000000000000000000000000000000000000000000000000000000000000000000000000000000000000000000001CFC63
:425C0A00000000000000000000000000000000000000000000000000000000000000000000000000000000000000000000000000000000000000000000000000000000003CFE1E
:425C4C00000000000000001000020000000000000000000000000000000000000000000000000000000000000000000000000000000000000000000000000000000000000CFEFA
:425C8E00000000000000000000000000000000000000000000000000000000000000000000000000000000000000000000000000000000000000000000000000000000003CFE9A
:425CD000000000000000000000000000000000000000000000000000000000000000000000000000000000000000000000000000000000000000000000000000000000002DFF66
:425D120000000000000000000804000000000000000000000000000000000000000000000000000000000000000000000000000000000000000000000000000000000000F4FE51
:425D54000000000000000000400010000000000000000000000000000000000000000000000000000000000000000000000000000000000000000000000000000000000028FE97
:425D9600000000000000000002000000000000000000000000000000000000000000000000000000000000000000000000000000000000000000000000000000000000003CFC91
:425DD800000000000000000000000000000000000000000000000000000000000000000000000000000000000000000000000000000000000000000000000000000000003CFE4F
:425E1A00000000000000000000000000000000000000000000000000000000000000000000000000000000000000000000000000000000000000000000000000000000003CFE0C
:425E5C0000000000000000000080000000000000000000000000000000000000000000000000000000000000000000000000000000000000000000000000000000000000B4FED2
:425E9E004000000000000000008000000000000000000000000000000000000000000000000000000000000000000000000000000000000000000000000000000000004096FC30
:425EE0000000000000000000000000000000000000000000000000000000000000000000000000000000000000000000000000000000000000000000000000000000004069FFD8
:425F22004000000000000000000A01000000000000000000000000000000000000000000000000000000000000000000000000000050000000000000000000000000000098FF0B
:425F640000000000000000100922020085045115000040000000000000000000000000000000000000000000000000000004000000184002001402010008040000000000E4FE2C
:425FA60000000000000000000000000002002008000010000000000000000000000000000000000000000000000000000000000000080000001000000000000000000000A4FCC7
:425FE800000000000000000800010000004000000000000000000000000000000000000000000000000000000000000000040000000480000000000100000400000000003CFF66
:42602A00000000000000000000000000000000000000000000000000000000000000000000000000000000000000000000000000000000000000000000000000000000003CFEFA
:42606C00000000000000000000000000000000000000000000000000000000000000000000000000000000000000000000000000000000000000000000000000000000003CFEB8
:4260AE00100000000000000000008000000000000000000000000000000000000000000000000000000000000000000000000000000000000000000000000000000000009EFD85
:4260F000000000000000000000000001000000000000000000000000000000000000000000000000000000000000000000000000000000000000000000000000000000003CFF32
:4261320000000000000000000000400002000080000000000000000000000000000000000000000000000000000000000000000000000000000000000000000000000000D4FE97
:42617400000000000000000000000000000000000000000000000000000000000000000000000000000000000000000000000000000000000000000000000000000000003CFEAF
:4261B600000000000000000000000000000000000000000000000000000000000000000000000000000000000000000000000000000000000000000000000000000000003CFE6D
:4261F800000000000000000000000000000000000000000000000000000000000000000000000000000000000000000000000000000000000000000000000000000000003CFE2B
:42623A0000000000000000000480001000000000000000000000000000000000000000000000000000000000000000000000000000000000000000000000000000000000E0FFAF
:42627C000000000000000000000008000000000000000000000000000000000000000000000000000000000000000000000000000000000000000000000000000000000034FEA6
:4262BE000000000000000000000000000000000000000000000000000000000000000000000000000000000000000000000000000000000000000000000000000000004078FEE8
:42630000000000000000000000000020000000000000000000000000000000000000000000000000000000000000000000000000000000000000000000000000000000001CFC23
:426342000000000000C04000000000000000000000000000000000000000000000000000000000000000000000000000000000000000000000000000000000000000000074FEA7
:42638400000000000000000000000000000000000000000000000000000000000000000000000000000000000000000000000000000000000000000000000000000000003CFE9D
:4263C6000000000000F00000000000000000000000000000000000000000000000000000000000000000000000000000000000000000000000000000000000000000000000FDA8
:4264080000000000001084000000000000000000000000000000000000000000000000000000000000000000000000000000000000000000000000000000000000000000E4FFDB
:42644A00000000000000000000000000000000000000000000000000000000000000000000000000000000000000000000000000000000000000000000000000000000003CFED6
:42648C000000000000F00000000000000000000000000000000000000000000000000000000000000000000000000000000000000000000000000000000000000000000000FDE1
:4264CE00000000000000000000000000000000000000000000000000000000000000000000000000000000000000000000000000000000000000000000000000000000003CFE52
:426510000000000000C00000000000000000000000000000000000000000000000000000000000000000000000000000000000000000000000000000000000000000000030FE5B
:426552000000008000000000000000000000000000000000000000000000000000000000000000000000000000000000000000000000000000000000000000000000000096FCF5
:42659400000000000000000000000000000000000000000000000000000000000000000000000000000000000000000000000000000000000000000000000000000000003CFE8B
:4265D6000000000006000000000000000000000000000000000000000000000000000000000000000000000000000000000000000000000000000000000000000000000018FC69
:426618000800000040040000000000000000000000000000000000000000000000000000000000000000000000000000000000000000000000000000000000000000008021FF54
:42665A0000000000260100000000000000000000000000000000000000000000000000000000000000000000000000000000000000000000000000000000000000000080B0FDAA
:42669C0000000080010000000000000000000000000000000000000000000000000000000000000000000000000000000000000000000000000000000000000000000000A4FF98
:4266DE00040000000601000000000000000000000000000000000000000000000000000000000000000000000000000000000000000000000000000000000000000000006BFE06
:426720000000000016000000000000000000000000000000000000000000000000000000000000000000000000000000000000000000000000000000000000000000000008FC1D
:426762000000040000C018000000000000000000000000000000000000000000000000000000000000000000000000000000000000000000000000000000000000000000F4FF26
:4267A400000000000000000000000000000000000000000000000000000000000000000000000000000000000000000000000000000000000000000000000000000000003CFE79
:4267E6000000000000F04000000000000000000000000000000000000000000000000000000000000000000000000000000000000000000000000000000000000000000044FD00
:42682800040030120010020000000000000000000000000000000000000000000000000000000000000000000000000000000000000000000000000000000000000000004DFC8D
:42686A000C000041000000000000000000000000000000000000000000000000000000000000000000000000000000000000000000000000000000000000000000000000A8FEF9
:4268AC0000003C0000F000000000000000000000000000000000000000000000000000000000000000000000000000000000000000000000000000000000000000000000FCFE84
:4268EE000800302000000000000000000000000000000000000000000000000000000000000000000000000000000000000000000000000000000000000000000000008004FF8D
:426930000000300100C00000000000000000000000000000000000000000000000000000000000000000000000000000000000000000000000000000000000000000000010FD27
:426972000000040016C018000000000000000000000000000000000000000000000000000000000000000000000000000000000000000000000000000000000000000000E2FF10
:4269B400000000000002000000000000000000000000000000000000000000000000000000000000000000000000000000000000000000000000000000000000000000003CFC67
:4269F6000000308007F28000000000000000000000000000000000000000000000000000000000000000000000000000000000000000000000000000000000000000000004FF33
:426A3800080000921010000000000000000000000000000000000000000000000000000000000000000000000000000000000000000000000000000000000000000000808DFF56
:426A7A0000003012000000000000000000000000000000000000000000000000000000000000000000000000000000000000000000000000000000000000000000000080A4FC78
:426ABC0000000C8007F00000000000000000000000000000000000000000000000000000000000000000000000000000000000000000000000000000000000000000000070FEA7
:426AFE00040030000000000000000000000000000000000000000000000000000000000000000000000000000000000000000000000000000000000000000000000000007FFEA5
:426B40000000302006C00000000000000000000000000000000000000000000000000000000000000000000000000000000000000000000000000000000000000000000024FDDC
:426B82000000048000C018180800000000000000000000000000000000000000000000000000000000000000000000000000000000000000000000000000000000000000CEFD8A
:426BC400000000000000000000000000000000000000000000000000000000000000000000000000000000000000000000000000000000000000000000000000000000003CFE55
:426C06000000000000F0001E00000000000000000000000000000000000000000000000000000000000000000000000000000000000000000000000000000000000000003CFF03
:426C48000800301246128482020000000000000000000000000000000000000000000000000000000000000000000000000000000000000000000000000000000000008029FCBB
:426C8A0000000006100000000000000000000000000000000000000000000000000000000000000000000000000000000000000000000000000000000000000000000080C4FE70
:426CCC0000003C8007F4001E000000000000000000000000000000000000000000000000000000000000000000000000000000000000000000000000000000000000000038FF7A
:426D0E00040030200602000000000000000000000000000000000000000000000000000000000000000000000000000000000000000000000000000000000000000000005BFC90
:426D50000000300226C0001800000000000000000000000000000000000000000000000000000000000000000000000000000000000000000000000000000000000000003CFF96
:426D92001000048000C002000000000000000000000000000000000000000000000000000000000000000000000000000000000000000000000000000000000000000000FEFD6E
:426DD4000000000000004000000000000000000000000000000000000000000000000000000000000000000000000000000000000000000000000000000000000000000078FEC7
:426E16000000300006F0800000000000000000000000000000000000000000000000000000000000000000000000000000000000000000000000000000000000000000009CFCFC
:426E58000400001240120000000000000000000000000000000000000000000000000000000000000000000000000000000000000000000000000000000000000000008095FD7E
:426E9A0004003011460000000000000000000000000000000000000000000000000000000000000000000000000000000000000000000000000000000000000000000080B0FEFD
:426EDC0000000C8001F20000000000000000000000000000000000000000000000000000000000000000000000000000000000000000000000000000000000000000000054FEA3
:426F1E000C003000060000000000000000000000000000000000000000000000000000000000000000000000000000000000000000000000000000000000000000000000DBFC18
:426F60000000B02046C1000000000000000000000000000000000000000000000000000000000000000000000000000000000000000000000000000000000000000000006CFCB0
:426FA2000000048000C00200000000000000000000000000000000000000000000000000000000000000000000008031000000000000000000000000000000000000000056FD63
:426FE4000000000000004000000000000000000000000000000000000000000000000000000000000000000000000000000000000000000000000000000000000000000078FEB5
:427026000000300000F0000000000000000000000000000000000000000000000000000000000000000000000000E08100000000000000000000000000000000000000006CFD3E
:427068000400002200108400000000000000000000000000000000000000000000000000000000000000000000002004000000000000000000000000000000000000008019FE71
:4270AA000C00B00006010000000000000000000000000000000000000000000000000000000000000000000000000000000000000000000000000000000000000000008068FEFB
:4270EC0000000C8807F0000000000000000000000000000000000000000000000000000000000000000000000000E00100000000000000000000000000000000000000002CFDCD
:42712E000800300006000000000000000000000000000000000000000000000000000000000000000000000000000000000000000000000000000000000000000000008031FE32
:427170000000300A06C0000000000000000000000000000000000000000000000000000000000000000000000000800100000000000000000000000000000000000000001CFE42
:4271B2000000048000100018080000000000000000001000000000000000000000000000000000000000000000000000000000000000000000000000000000000000000070FE69
:4271F400000000000000000000000000000000000000000000000000000000000000000000000000000000000000000000000000000000000000000000000000000000003CFE1F
:42723600000030000000001E100000000000000000000000000000000000000000000000000000000000000000000000000000000000000000000000000000000000000020FE9A
:42727800040000220000000200000000000000000000000000000000000000000000000000000000000000000000000000000000000000000000000000000000000000006DFF40
:4272BA000C00300986C0100000000000000000000000C010000000000000000000000000000000000000000000000000000000000000000000000000000000000000000028FE01
:4272FC0000000C8007F0001E00000000000000000000F000000000000000000000000000000000000000000000000000000000000000000000000000000000000000000080FF40
:42733E0008003008000020000000000000000000000000400000000000000000000000000000000000000000000000000000000000000000000000000000000000000080C4FF2A
:427380000000B0004001001800000000000000000000000000000000000000000000000000000000000000000000000000000000000000000000000000000000000000005CFC6A
:4273C200000000000000000000000000000000000000000000000000000000000000000000000000000000000000000000000000000000000000000000000000000000003CFE4F
:427404002000048000100002400008000120000480001000024000080001200004000000000010000240000800012000048000100002400008000120000480001000020034FCE4
:42744600000000000000000000000000000000000000000000000000000000000000000000000000000000000000000000000000000000000000000000000000000000003CFECA
:42748800280004800010000240000800012000048000100002400008000120000400000000001000024000080001200004800010000240000800012000048000100002802DFDDE
:4274CA0000000000048000100000000000000000000000000000000000000000000000000000000000000000000000010000000000000000000000000000000000000080B8FFB4
:42750C00200004000000000040000800012000048000100002400008000120000400000000001000024000080001000004800010000240000800012000048000100002008CFD34
:42754E0004000000000000000000000000000000000000000000000000000000000000000000000000000000000000000000000000000000000000000000000000000080E5FF93
:427590002000048000100002400008000120000480001000024000080001200004000000000010000240000800012000048000100002400008000120000480001000020034FC57
:4275D200000000000000000000000000000000000000000000000000000000000000000000000000000000000000000000000000000000000000000000000000000000003CFE3D
:42761400000000000000000000000000000000000000000000000000000000000000000000000000000000000000000000000000000000000000000000000000000000003CFEFA
:427656000000200006000000000000000000000000000000000000000000000000000000000000000000000000000000000000000000000000000000000000000000000038FE96
:42769800000000000000000000000000000000000000000000000000000000000000000000000000000000000000000000000000000000000000000000000000000000003CFE76
:4276DA00000000000000000000000000000000000000000000000000000000000000000000000000000000000000000000000000000000000000000000000000000000C0F0FEC0
:42771C00000000000000000000000000000000000000000000000000000000000000000000000000000000000000000000000000000000000000000000000000000000003CFEF1
:42775E0000000000000000000000000000000000000000000000000000000000000000000000000000000000000080000000000000000000000000000000000000000000B4FEB7
:4277A0000000000000004000000000000000000000000000000000000000000000000000000000000000000000000000000000000000000000000000000000000000000078FEF1
:4277E2000000000000400000000000000000000000000000000000000000000000000000000000000000000000002000000000000000000000000000000000000000000038FCD1
:42782400000000000000000200000000000000000000000000000000000000000000000000000000000000000000000000000000000000000000000000000000000000001CFC08
:42786600000000000000000000000000000000000000000000000000000000000000000000000000000000000000000000000000000000000000000000000000000000003CFEA6
:4278A800000000000000000000000000000000000000000000000000000000000000000000000000000000000000000000000000000000000000000000000000000000C0D2FC10
:4278EA000000000000000000000000000004000000000000000000000000000000000000000000000000000000000000200000000000080000000000000000000000000090FCA4
:42792C000000000000400000000000000000000000000000000000000000000000000000000000000000000000000000000400000000000000000000000000000000000078FE5F
:42796E0000000000A01014000000000000040000000000000000000000000000000000000000000000000000000000000820000000000800000000000000000000000000C8FC1B
:4279B0000001100022C00400000000000000000000000000000000000000000000000000000000000000000000000000200000000000000000000000000000000000000050FE30
:4279F2000000200004800000000000000000000000000000000000000000000000000000000000000000000000000000000000000000000000000000000000000000000010FCA3
:427A34000001000000400000000000000000000000000000000000000000000000000000000000000000000000000000200000000000000000000000000000000000000008FDAA
:427A7600000000000000000000000000000000000000000000000000000000000000000000000000000000000000000000000000000000000000000000000000000000003CFE94
:427AB8000000000004800000000000000000000000000000000000000000000000000000000000000000000000000000000000000000000000000000000000000000000030FEDA
:427AFA00000000000000000000000000000000000000000000000000000000000000000000000000000000000000000000000000000000000000000000000000000000003CFE10
:427B3C00000000000000024000000000000000000000000000000000000000000000000000000000000000000000000000000000000000000000000000000000000000005CFE6B
:427B7E00000000000000000000000000000000000000000000000000000000000000000000000000000000000000000000000000000000000000000000000000000000001EFCAB
:427BC000000000000000000000000000000000000000000000000000000000000000000000000000000000000000000000000000000000000000000000000000000000003CFE49
:427C0200000000000010000000000000000000000000000000000000000000000000000000000000000000000000000000000000000000000000000000000000000000002CFF05
:427C4400000000000000000000000000000000000000000000000000000000000000000000000000000000000000000000000000000000000000000000000000000000003CFEC4
:427C8600000000000000000000000000000000000000000000000000000000000000000000000000000000000000000000000000000000000000000000000000000000003CFE82
:427CC800000000000000000000000000000000000000000000000000000000000000000000000000000000000000000000000000000000000000000000000000000000003CFE40
:427D0A000000040000000000000000000000000000000000000000000000000000000000000000000000000000000000000000000000000000000000000000000000000078FEBD
:427D4C0000000080001000000000000000000000000010000000000000000000000000000000000000000000000000000000000000000000000000000000000000000000A4FEB3
:427D8E000000000008000000000000000000000000000000000000000000000000000000000000000000000000000000000000000000000000000000000000000000000034FE79
:427DD00000001840000000000000000000000000000000000000000000000000000000000000000000000000000000000000000000000000000000000000000000000000E0FF3A
:427E1200000000000000000000000000000000000000000000000000000000000000000000000000000000000000000000000000000000000000000000000000000000003CFEF4
:427E54000000000000000000000000000000000000000000000000000000000000000000000000000000000000000000000000000000000000000000000000000000004078FE36
:427E9600000000000000000000000000000000000000000000000000000000000000000000000000000000000000000000000000000000000000000000000000000000003CFE70
:427ED800000000000001000000000000000000000000000000000000000000000000000000000000000000000000000000000000000000000000000000000000000000001EFD4C
:427F1A00400000000040000000000000000000000000000000000000000000000000000000000000000000000000000000000000000000000000000000000000000000C092FC57
:427F5C00000000000000200000000000000000000000000000000000000000000000000000000000000000000000000000000000000000000000000000000000000000002DFD99
:427F9E004000A00000208000000000000000000006000000000000000000000000000000000000000000000000008000000000000000000000000000000000000000000054FC4B
:427FE00020020000C111480C8044200000000000000CA000000000000000000000000000000000000000000000000001200400800000000000000000000000000000000004FEE0
:4280220000000000800000040000100000000000000000000000000000000000000000000000000000000000000000000000000000000000000000000000000000000000A8FEE2
:4280640000000000000100000000020000000000000210000000000000000000000000000000000000000000000040000804002000000000000000000000000000000000B0FCAD
:4280A600000000100000000000000000000000000000000000000000000000000000000000000000000000000000000000000000000000000000000000000000000000003CFF4D
:4280E800120000000000000000000000000000000000200000000000000000000000000000000000000000000000000000000000000000000000000000000000000000407AFF6B
:42812A000000800001000000000000000000000000000000000000000000000000000000000000000000000000000000000000000000000000000000000000000000000024FF6F
:42816C000000000C000000000000000000000000000000000000000000000000000000000000000000000000000000000000000000000000000000000000000000000000FCFECB
:4281AE00000000000020000400000000000000000000000000000000000000000000000000000000000000000000000000000000000000000000000000000000000000003AFE33
:4281F000000000000000000000000000000000000000000000000000000000000000000000000000000000000000000000000000000000000000000000000000000000003CFE13
:42823200000000000000000000000000000000000000000000000000000000000000000000000000000000000000000000000000000000000000000000000000000000003CFED0
:42827400000000000000000000000000000000000000000000000000000000000000000000000000000000000000000000000000000000000000000000000000000000003CFE8E
:4282B60000000008000100000000000000000000000000000000000000000000000000000000000000000000000000000000000000000000000000000000000000000000ADFED2
:4282F800000000000000000000000000000000000000000000000000000000000000000000000000000000000000000000000000000000000000000000000000000000003CFE0A
:42833A00000000000000000000000000000000000000000000000000000000000000000000000000000000000000000000000000000000000000000000000000000000003CFEC7
:42837C00000000000000000000000000000000000000000000000000000000000000000000000000000000000000000000000000000000000000000000000000000000003CFE85
:4283BE00000000000000000000000000000000000000000000000000000000000000000000000000000000000000000000000000000000000000000000000000000000003CFE43
:42840000000000000000000000000000000000000000000000000000000000000000000000000000000000000000000000000000000000000000000000000000000000003CFE00
:42844200000000000000000000000000000000000000000000000000000000000000000000000000000000000000000000000000000000000000000000000000000000003CFEBE
:42848400000000000000000000000000000000000000000000000000000000000000000000000000000000000000000000000000000000000000000000000000000000003CFE7C
:4284C600000000000000000000000000000000000000000000000000000000000000000000000000000000000000000000000000000000000000000000000000000000003CFE3A
:42850800000000000000000000000000000000000000000000000000000000000000000000000000000000000000000000000000000000000000000000000000000000003CFEF7
:42854A00000000000000000000000000000000000000000000000000000000000000000000000000000000000000000000000000000000000000000000000000000000003CFEB5
:42858C00000000000000000000000000000000000000000000000000000000000000000000000000000000000000000000000000000000000000000000000000000000003CFE73
:4285CE00000000000000000000000000000000000000000000000000000000000000000000000000000000000000000000000000000000000000000000000000000000001EFC51
:42861000000000000000000000000000000000000000000000000000000000000000000000000000000000000000000000000000000000000000000000000000000000003CFEEE
:42865200000000000000000000000000000000000000000000000000000000000000000000000000000000000000000000000000000000000000000000000000000000003CFEAC
:428694000800000000000000000000000000000000000000000000000000000000000000000000000000000000000000000000000000000000000000000000000000008025FFF8
:4286D60000000000000000000000000000000000000000000000000000000000000000000000000000000000000000000000000000000000000000000000000000000080B4FE30
:42871800000000000000000000000000000000000000000000000000000000000000000000000000000000000000000000000000000000000000000000000000000000002DFFF3
:42875A00040000000000000000000000000000000000000000000000000000000000000000000000000000000000000000000000000000000000000000000000000000006DFF6D
:42879C00000000000000000000000000000000000000000000000000000000000000000000000000000000000000000000000000000000000000000000000000000000001EFC81
:4287DE00000000000000000000000000000000000000000000000000000000000000000000000000000000000000000000000000000000000000000000000000000000003CFE1F
:42882000000000000000000000000000000000000000000000000000000000000000000000000000000000000000000000000000000000000000000000000000000000003CFEDC
:42886200000000000000000000000000000000000000000000000000000000000000000000000000000000000000000000000000000000000000000000000000000000003CFE9A
:4288A400040000000000000000000000000000000000000000000000000000000000000000000000000000000000000000000000000000000000000000000000000000006DFF22
:4288E6000C000000000000000000000000000000000000000000000000000000000000000000000000000000000000000000000000000000000000000000000000000000FCFE4A
:42892800000000000000000000000000000000000000000000000000000000000000000000000000000000000000000000000000000000000000000000000000000000003CFED3
:42896A000800000000000000000000000000000000000000000000000000000000000000000000000000000000000000000000000000000000000000000000000000008034FE11
:4289AC00000000000000000000000000000000000000000000000000000000000000000000000000000000000000000000000000000000000000000000000000000000003CFE4F
:4289EE00000000000000000000000000000000000000000000000000000000000000000000000000000000000000000000000000000000000000000000000000000000001EFC2D
:428A3000000000000000000000000000000000000000000000000000000000000000000000000000000000000000000000000000000000000000000000000000000000003CFECA
:428A7200000000000000000000000000000000000000000000000000000000000000000000000000000000000000000000000000000000000000000000000000000000003CFE88
:428AB4000800000000000000000000000000000000000000000000000000000000000000000000000000000000000000000000000000000000000000000000000000008025FFD4
:428AF60000000000000000000000000000000000000000000000000000000000000000000000000000000000000000000000000000000000000000000000000000000080B4FE0C
:428B3800000000000000000000000000000000000000000000000000000000000000000000000000000000000000000000000000000000000000000000000000000000002DFFCF
:428B7A00040000000000000000000000000000000000000000000000000000000000000000000000000000000000000000000000000000000000000000000000000000006DFF49
:428BBC00000000000000000000000000000000000000000000000000000000000000000000000000000000000000000000000000000000000000000000000000000000001EFC5D
:428BFE00000000000000000000000000000000000000000000000000000000000000000000000000000000000000000000000000000000000000000000000000000000001EFC1B
:428C4000000000000000000000000000000000000000000000000000000000000000000000000000000000000000000000000000000000000000000000000000000000003CFEB8
:428C8200000000000000000000000000000000000000000000000000000000000000000000000000000000000000000000000000000000000000000000000000000000003CFE76
:428CC40004000000000000000000000000000000000000000000000000000000000000000000000000000000000000000000000000000000000000000000000000000080E5FF06
:428D06000C00000000000000000000000000000000000000000000000000000000000000000000000000000000000000000000000000000000000000000000000000008074FE2D
:428D4800000000000000000000000000000000000000000000000000000000000000000000000000000000000000000000000000000000000000000000000000000000002DFFBD
:428D8A0008000000000000000000000000000000000000000000000000000000000000000000000000000000000000000000000000000000000000000000000000000000ADFFF3
:428DCC00000000000000000000000000000000000000000000000000000000000000000000000000000000000000000000000000000000000000000000000000000000001EFC4B
:428E0E00000000000000000000000000000000000000000000000000000000000000000000000000000000000000000000000000000000000000000000000000000000001EFC08
:428E5000000000000000000000000000000000000000000000000000000000000000000000000000000000000000000000000000000000000000000000000000000000003CFEA6
:428E9200000000000000000000000000000000000000000000000000000000000000000000000000000000000000000000000000000000000000000000000000000000003CFE64
:428ED4000800000000000000000000000000000000000000000000000000000000000000000000000000000000000000000000000000000000000000000000000000008025FFB0
:428F160000000000000000000000000000000000000000000000000000000000000000000000000000000000000000000000000000000000000000000000000000000080B4FEE7
:428F5800000000000000000000000000000000000000000000000000000000000000000000000000000000000000000000000000000000000000000000000000000000002DFFAB
:428F9A00040000000000000000000000000000000000000000000000000000000000000000000000000000000000000000000000000000000000000000000000000000006DFF25
:428FDC00000000000000000000000000000000000000000000000000000000000000000000000000000000000000000000000000000000000000000000000000000000001EFC39
:42901E00000000000000000000000000000000000000000000000000000000000000000000000000000000000000000000000000000000000000000000000000000000001EFCF6
:42906000000000000000000000000000000000000000000000000000000000000000000000000000000000000000000000000000000000000000000000000000000000003CFE94
:4290A200000000000000000000000000000000000000000000000000000000000000000000000000000000000000000000000000000000000000000000000000000000003CFE52
:4290E40004000000000000000000000000000000000000000000000000000000000000000000000000000000000000000000000000000000000000000000000000000080E5FFE2
:429126000C00000000000000000000000000000000000000000000000000000000000000000000000000000000000000000000000000000000000000000000000000008074FE09
:42916800000000000000000000000000000000000000000000000000000000000000000000000000000000000000000000000000000000000000000000000000000000002DFF99
:4291AA0008000000000000000000000000000000000000000000000000000000000000000000000000000000000000000000000000000000000000000000000000000000ADFFCF
:4291EC00000000000000000000000000000000000000000000000000000000000000000000000000000000000000000000000000000000000000000000000000000000001EFC27
:42922E00000000000000000000000000000000000000000000000000000000000000000000000000000000000000000000000000000000000000000000000000000000003CFEC4
:42927000000000000000000000000000000000000000000000000000000000000000000000000000000000000000000000000000000000000000000000000000000000003CFE82
:4292B200000000000000000000000000000000000000000000000000000000000000000000000000000000000000000000000000000000000000000000000000000000003CFE40
:4292F400040000000000000000000000000000000000000000000000000000000000000000000000000000000000000000000000000000000000000000000000000000006DFFC8
:429336000C000000000000000000000000000000000000000000000000000000000000000000000000000000000000000000000000000000000000000000000000000000FCFEEF
:42937800000000000000000000000000000000000000000000000000000000000000000000000000000000000000000000000000000000000000000000000000000000003CFE79
:4293BA000800000000000000000000000000000000000000000000000000000000000000000000000000000000000000000000000000000000000000000000000000008034FEB7
:4293FC00000000000000000000000000000000000000000000000000000000000000000000000000000000000000000000000000000000000000000000000000000000003CFEF5
:42943E00000000000000000000000000000000000000000000000000000000000000000000000000000000000000000000000000000000000000000000000000000000001EFCD2
:429480002000048000100002400008000120000480001000024000080001200004000000000010000240000800012000048000100002400008000120000480001000020034FC48
:4294C200000000000000000000000000000000000000000000000000000000000000000000000000000000000000000000000000000000000000000000000000000000003CFE2E
:42950400280004800010000240000800012000048000100002400008000120000400000000001000024000080001200004800010000240000800012000048000100002802DFD41
:4295460000000000000000000000000000000000000000000000000000000000000000000000000000000000000000000000000000000000000000000000000000000080B4FEB1
:429588002000048000100002400008000120000480001000024000080001200004000000000010000240000800012000048000100002400008000120000480001000020025FD4D
:4295CA00040000000000000000000000000000000000000000000000000000000000000000000000000000000000000000000000000000000000000000000000000000006DFFEF
:42960C002000048000100002400008000120000480001000024000080001200004000000000010000240000800012000048000100002400008000120000480001000020016FED6
:42964E00000000000000000000000000000000000000000000000000000000000000000000000000000000000000000000000000000000000000000000000000000000003CFEA0
:42969000000000000000000000000000000000000000000000000000000000000000000000000000000000000000000000000000000000000000000000000000000000003CFE5E
:4296D200000000000000000000000000000000000000000000000000000000000000000000000000000000000000000000000000000000000000000000000000000000003CFE1C
:42971400000000000000000000000000000000000000000000000000000000000000000000000000000000000000000000000000000000000000000000000000000000003CFED9
:42975600000000000000000000000000000000000000000000000000000000000000000000000000000000000000000000000000000000000000000000000000000000003CFE97
:429798000000000000000000000000000000000000000000000000000000000000000000000000000000000000000000000000000000000000000000000000000000004078FED9
:4297DA00000000000000000000000000000000000000000000000000000000000000000000000000000000000000000000000000000000000000000000000000000000003CFE13
:42981C00000000000000000000000000000000000000000000000000000000000000000000000000000000000000000000000000000000000000000000000000000000003CFED0
:42985E00000000000000000000000000000000000000000000000000000000000000000000000000000000000000000000000000000000000000000000000000000000003CFE8E
:4298A000000000000000000000000000000000000000000000000000000000000000000000000000000000000000000000000000000000000000000000000000000000003CFE4C
:4298E200000000000000000000000000000000000000000000000000000000000000000000000000000000000000000000000000000000000000000000000000000000003CFE0A
:4299240000000000000000000000000000000000000000000000000000000000000000000000000000000000000000000000000000000000000000000000000000000080B4FECF
:42996600000000000000000000000000000000000000000000000000000000000000000000000000000000000000000001000000000000000000000000000000000000003CFF83
:4299A800000000000000000000000000000000000000000010000000000000000000000000000000000000000000000000000000000000000000000000000000000000002CFF42
:4299EA0000000000000000000000000000000000000000000200000000000000000000000000000000000000000000800000000000000000000000000000000000000000BCFC01
:429A2C0000000000000000000000000000000000000000000000000000000000000000000000000000000000000080000000000000000000000000000000000000000000B4FEC6
:429A6E00000000000000000000000000000000000000000000000000000000000000000000000000000000000000000100000000000000000000000000000000000000002CFF8A
:429AB0000200000000000000000000000000000000000000000000000000000000000000000000000000000000000000000000000000000000000000000000000000004058FEDC
:429AF200000000000000000000000000000000000000000000000000000000000000000000000000000000000000000000000000000000000000000000000000000000003CFEF8
:429B3400000000000000000000000000000000000000000000000000000000000000000000000000000000000000000000000000000000000000000000000000000000003CFEB5
:429B7600000000000000000000000000000000000000000000000000000000000000000000000000000000000000000000000000000000000000000000000000000000003CFE73
:429BB800000000000000000000000000000000000000000000000000000000000000000000000000000000000000000000000000000000000000000000000000000000003CFE31
:429BFA00000000000000000000000000000000000000000000000000000000000000000000000000000000000000000000000000000000000000000000000000000000003CFEEF
:429C3C0000000000000000000000000000000000000000000000000000000000000000000000000000000000000000000000000000000000000000000000000000000080B4FEB4
:429C7E00000000000000000000000000000000000000000000000000000000000000000000000000000000000000000000000000000000000000000000000000000000001EFC8A
:429CC000000000000000000000000000000000000000000000000000000000000000000000000000000000000000000000000000000000000000000000000000000000003CFE28
:429D0200000000000000000000000000000000000000000000000000000000000000000000000000000000000000000000000000000000000000000000000000000000003CFEE5
:429D4400000000000000000000000000000000000000000000000000000000000000000000000000000000000000000000000000000000000000000000000000000000003CFEA3
:429D8600000000000000000000000000000000000000000000000000000000000000000000000000000000000000000000000000000000000000000000000000000000003CFE61
:429DC800000000000000000000000000000000000000000000000000000000000000000000000000000000000000000000000000000000000000000000000000000000003CFE1F
:429E0A000000000000000000000000000000000000000000000000000000000000000000000000000000000000000000000000000000000000000000000000000000004078FE60
:429E4C00000000000000000000000000000000000000000000000000000000000000000000000000000000000000000000000000000000000000000000000000000000003CFE9A
:429E8E00000000000000000000000000000000000000000000000000000000000000000000000000000000000000000000000000000000000000000000000000000000003CFE58
:429ED000000000000000000000000000000000000000000000000000000000000000000000000000000000000000000000000000000000000000000000000000000000002DFF24
:429F1200000000000000000000000000000000000000000000000000000000000000000000000000000000000000000000000000000000000000000000000000000000003CFED3
:429F5400000000000000000000000000000000000000000000000000000000000000000000000000000000000000000000000000000000000000000000000000000000003CFE91
:429F9600000000000000000000000000000000000000000000000000000000000000000000000000000000000000000000000000000000000000000000000000000000C0D2FCFB
:429FD8000000000000000000000000000000000000000000001000000000000000000000000000000000000000000000000000000000000000000000000000000000004069FE90
:42A01A0000000000000000000000C000800103600600800100100000000000000000000000000000000000000000000000000000000000000000000000000000000000009CFC31
:42A05C000000000000800000000000000000000000000000000042000000000000000000000000000000000000000000000000000000000000000000000000000000000054FCB0
:42A09E00000000000000000000000000000000000000000000000000000000000000000000000000000000000000000000000000000000000000000000000000000000003CFE46
:42A0E000000000000020000000000000000000000000000000000202000000000000000000000000000000000000000000000000000000000000000000000000000000003CFCE2
:42A12200100000000000000000000000000000000000000000000000000000000000000000000000000000000000000000000000000000000000000000000000000000001EFDD0
:42A16400000000000000000000000000000000000000000000000000000000000000000000000000000000000000000000000000000000000000000000000000000000003CFE7F
:42A1A600000000000000000000000000000000000000000000000000000000000000000000000000000000000000000000000000000000000000000000000000000000003CFE3D
:42A1E80004000000000000000000000000000000000000000000000000000000000000000000000000000000000000000000000000000000000000000000000000000080F4FEBF
:42A22A00040000000000000000000000000000000000000000000000000000000000000000000000000000000000000000000000000000000000000000000000000000400BFDA6
:42A26C00000000000000000000000000000000000000000000000000000000000000000000000000000000000000000000000000000000000000000000000000000000003CFE76
:42A2AE00000000000000000000000000000000000000000000000000000000000000000000000000000000000000000000000000000000000000000000000000000000003CFE34
:42A2F000000000000000000000000000000000000000000000000000000000000000000000000000000000000000000000000000000000000000000000000000000000001EFC12
:42A33200000000000000000000000000000000000000000000000000000000000000000000000000000000000000000000000000000000000000000000000000000000003CFEAF
:42A37400000000000000000000000000000000000000000000000000000000000000000000000000000000000000000000000000000000000000000000000000000000003CFE6D
:42A3B600000000000000000000000000000000000000000000000000000000000000000000000000000000000000000000000000000000000000000000000000000000003CFE2B
:42A3F800000000000000000000000000000000000000000000000000000000000000000000000000000000000000000000000000000000000000000000000000000000003CFEE9
:42A43A00000000000000000000000000000000000000000000000000000000000000000000000000000000000000000000000000000000000000000000000000000000003CFEA6
:42A47C00000000000000000000000000000000000000000000000000000000000000000000000000000000000000000000000000000000000000000000000000000000003CFE64
:42A4BE00000000000000000000000000000000000000000000000000000000000000000000000000000000000000000000000000000000000000000000000000000000003CFE22
:42A50000000000000000000000000000000000000000000000000000000000000000000000000000000000000000000000000000000000000000000000000000000000003CFEDF
:42A54200000000000000000000000000000000000000000000000000000000000000000000000000000000000000000000000000000000000000000000000000000000003CFE9D
:42A58400000000000000000000000000000000000000000000000000000000000000000000000000000000000000000000000000000000000000000000000000000000003CFE5B
:42A5C600000000000000000000000000000000000000000000000000000000000000000000000000000000000000000000000000000000000000000000000000000000003CFE19
:42A60800000000000000000000000000000000000000000000000000000000000000000000000000000000000000000000000000000000000000000000000000000000003CFED6
:42A64A00000000000000000000000000000000000000000000000000000000000000000000000000000000000000000000000000000000000000000000000000000000001EFCB4
:42A68C00000000000000000000000000000000000000000000000000000000000000000000000000000000000000000000000000000000000000000000000000000000003CFE52
:42A6CE00000000000000000000000000000000000000000000000000000000000000000000000000000000000000000000000000000000000000000000000000000000003CFE10
:42A710000800000000000000000000000000000000000000000000000000000000000000000000000000000000000000000000000000000000000000000000000000008025FF5B
:42A7520000000000000000000000000000000000000000000000000000000000000000000000000000000000000000000000000000000000000000000000000000000080B4FE93
:42A79400000000000000000000000000000000000000000000000000000000000000000000000000000000000000000000000000000000000000000000000000000000002DFF57
:42A7D600040000000000000000000000000000000000000000000000000000000000000000000000000000000000000000000000000000000000000000000000000000006DFFD1
:42A81800000000000000000000000000000000000000000000000000000000000000000000000000000000000000000000000000000000000000000000000000000000001EFCE4
:42A85A00000000000000000000000000000000000000000000000000000000000000000000000000000000000000000000000000000000000000000000000000000000003CFE82
:42A89C00000000000000000000000000000000000000000000000000000000000000000000000000000000000000000000000000000000000000000000000000000000003CFE40
:42A8DE00000000000000000000000000000000000000000000000000000000000000000000000000000000000000000000000000000000000000000000000000000000003CFEFE
:42A92000040000000000000000000000000000000000000000000000000000000000000000000000000000000000000000000000000000000000000000000000000000006DFF85
:42A962000C000000000000000000000000000000000000000000000000000000000000000000000000000000000000000000000000000000000000000000000000000000FCFEAD
:42A9A400000000000000000000000000000000000000000000000000000000000000000000000000000000000000000000000000000000000000000000000000000000003CFE37
:42A9E6000800000000000000000000000000000000000000000000000000000000000000000000000000000000000000000000000000000000000000000000000000008034FE75
:42AA2800000000000000000000000000000000000000000000000000000000000000000000000000000000000000000000000000000000000000000000000000000000003CFEB2
:42AA6A00000000000000000000000000000000000000000000000000000000000000000000000000000000000000000000000000000000000000000000000000000000001EFC90
:42AAAC00000000000000000000000000000000000000000000000000000000000000000000000000000000000000000000000000000000000000000000000000000000003CFE2E
:42AAEE00000000000000000000000000000000000000000000000000000000000000000000000000000000000000000000000000000000000000000000000000000000003CFEEC
:42AB30000800000000000000000000000000000000000000000000000000000000000000000000000000000000000000000000000000000000000000000000000000008025FF37
:42AB720000000000000000000000000000000000000000000000000000000000000000000000000000000000000000000000000000000000000000000000000000000080B4FE6F
:42ABB400000000000000000000000000000000000000000000000000000000000000000000000000000000000000000000000000000000000000000000000000000000002DFF33
:42ABF600040000000000000000000000000000000000000000000000000000000000000000000000000000000000000000000000000000000000000000000000000000006DFFAD
:42AC3800000000000000000000000000000000000000000000000000000000000000000000000000000000000000000000000000000000000000000000000000000000001EFCC0
:42AC7A00000000000000000000000000000000000000000000000000000000000000000000000000000000000000000000000000000000000000000000000000000000003CFE5E
:42ACBC00000000000000000000000000000000000000000000000000000000000000000000000000000000000000000000000000000000000000000000000000000000003CFE1C
:42ACFE00000000000000000000000000000000000000000000000000000000000000000000000000000000000000000000000000000000000000000000000000000000003CFEDA
:42AD400008000000000000000000000000000000000000000000000000000000000000000000000000000000000000000000000000000000000000000000000000000000ADFF1D
:42AD8200000000000000000000000000000000000000000000000000000000000000000000000000000000000000000000000000000000000000000000000000000000003CFE55
:42ADC400000000000000000000000000000000000000000000000000000000000000000000000000000000000000000000000000000000000000000000000000000000003CFE13
:42AE060004000000000000000000000000000000000000000000000000000000000000000000000000000000000000000000000000000000000000000000000000000080F4FE94
:42AE4800000000000000000000000000000000000000000000000000000000000000000000000000000000000000000000000000000000000000000000000000000000003CFE8E
:42AE8A00000000000000000000000000000000000000000000000000000000000000000000000000000000000000000000000000000000000000000000000000000000003CFE4C
:42AECC00000000000000000000000000000000000000000000000000000000000000000000000000000000000000000000000000000000000000000000000000000000003CFE0A
:42AF0E00000000000000000000000000000000000000000000000000000000000000000000000000000000000000000000000000000000000000000000000000000000003CFEC7
:42AF5000040000000000000000000000000000000000000000000000000000000000000000000000000000000000000000000000000000000000000000000000000000006DFF4F
:42AF92000C000000000000000000000000000000000000000000000000000000000000000000000000000000000000000000000000000000000000000000000000000000FCFE77
:42AFD400000000000000000000000000000000000000000000000000000000000000000000000000000000000000000000000000000000000000000000000000000000003CFE01
:42B016000800000000000000000000000000000000000000000000000000000000000000000000000000000000000000000000000000000000000000000000000000008034FE3E
:42B05800000000000000000000000000000000000000000000000000000000000000000000000000000000000000000000000000000000000000000000000000000000003CFE7C
:42B09A00000000000000000000000000000000000000000000000000000000000000000000000000000000000000000000000000000000000000000000000000000000001EFC5A
:42B0DC00000000000000000000000000000000000000000000000000000000000000000000000000000000000000000000000000000000000000000000000000000000003CFEF8
:42B11E00000000000000000000000000000000000000000000000000000000000000000000000000000000000000000000000000000000000000000000000000000000003CFEB5
:42B160000C00000000000000000000000000000000000000000000000000000000000000000000000000000000000000000000000000000000000000000000000000008065FFBD
:42B1A20004000000000000000000000000000000000000000000000000000000000000000000000000000000000000000000000000000000000000000000000000000080F4FEF5
:42B1E400000000000000000000000000000000000000000000000000000000000000000000000000000000000000000000000000000000000000000000000000000000003CFEEF
:42B226000C00000000000000000000000000000000000000000000000000000000000000000000000000000000000000000000000000000000000000000000000000008065FFF6
:42B26800000000000000000000000000000000000000000000000000000000000000000000000000000000000000000000000000000000000000000000000000000000003CFE6A
:42B2AA00000000000000000000000000000000000000000000000000000000000000000000000000000000000000000000000000000000000000000000000000000000003CFE28
:42B2EC00000000000000000000000000000000000000000000000000000000000000000000000000000000000000000000000000000000000000000000000000000000003CFEE6
:42B32E00000000000000000000000000000000000000000000000000000000000000000000000000000000000000000000000000000000000000000000000000000000003CFEA3
:42B3700008000000000000000000000000000000000000000000000000000000000000000000000000000000000000000000000000000000000000000000000000000000ADFFE7
:42B3B200000000000000000000000000000000000000000000000000000000000000000000000000000000000000000000000000000000000000000000000000000000003CFE1F
:42B3F400000000000000000000000000000000000000000000000000000000000000000000000000000000000000000000000000000000000000000000000000000000003CFEDD
:42B4360004000000000000000000000000000000000000000000000000000000000000000000000000000000000000000000000000000000000000000000000000000080F4FE5E
:42B47800000000000000000000000000000000000000000000000000000000000000000000000000000000000000000000000000000000000000000000000000000000003CFE58
:42B4BA00100000000000000000000000000000000000000000000000000000000000000000000000000000000000000000000000000000000000000000000000000000003CFF05
:42B4FC002000048000100002400008000120000480001000024000080001200004000000000010000240000800012000048000100002400008000120000480001000020034FCAC
:42B53E00000000000000000000000000000000000000000000000000000000000000000000000000000000000000000000000000000000000000000000000000000000003CFE91
:42B580002C0004800010000240000800012000048000100002400008000120000400000000001000024000080001200004800010000240000800012000048000100002806DFD61
:42B5C20004000000000000000000000000000000000000000000000000000000000000000000000000000000000000000000000000000000000000000000000000000080F4FED1
:42B604002000048000100002400008000120000480001000024000080001200004000000000010000240000800012000048000100002400008000120000480001000020034FCA2
:42B646000C00000000000000000000000000000000000000000000000000000000000000000000000000000000000000000000000000000000000000000000000000008065FFD2
:42B688002000048000100002400008000120000480001000024000080001200004000000000010000240000800012000048000100002400008000120000480001000020034FC1E
:42B6CA00000000000000000000000000000000000000000000000000000000000000000000000000000000000000000000000000000000000000000000000000000000003CFE04
:42B70C00000000000000000000000000000000000000000000000000000000000000000000000000000000000000000000000000000000000000000000000000000000003CFEC1
:42B74E00000000000000000000000000000000000000000000000000000000000000000000000000000000000000000000000000000000000000000000000000000000003CFE7F
:42B79000000000000000000000000000000000000000000000000000000000000000000000000000000000000000000000000000000000000000000000000000000000003CFE3D
:42B7D200000000000000000000000000000000000000000000000000000000000000000000000000000000000000000000000000000000000000000000000000000000003CFEFB
:42B81400000000000000000000000000000000000000000000000000000000000000000000000000000000000000000000000000000000000000000000000000000000003CFEB8
:42B85600000000000000000000000000000000000000000000000000000000000000000000000000000000000000000000000000000000000000000000000000000000003CFE76
:42B898000000000000000000000000000000000000000000000000000000000000000000000000000000000000000000000000000000000000000000000000000000008096FC5C
:42B8DA00000000000000000000000000000000000000000000000000000000000000000000000000000000000000000000000000000000000000000000000000000000003CFEF2
:42B91C00000000000000000000000000000000000000000000000000000000000000000000000000000000000000000000000000000000000000000000000000000000003CFEAF
:42B95E00000000000000000000000000000000000000000000000000000000000000000000000000000000000000000000000000000000000000000000000000000000003CFE6D
:42B9A000000000000000000000000000000000000000000000000000000000000000000000000000000000000000000000000000000000000000000000000000000000001EFC4B
:42B9E200000000000000000000000000000000000000000000000000000000000000000000000000000000000000000000000000000000000000000000000000000000003CFEE9
:42BA24000000000000000000000000000000000000000000004040000000000000000000000000000000000000000000000000000000000000000000000000000000000038FE2A
:42BA66000000000000000000000000000000000000000000004000020000000000000000000000000000000000000000000000000000000000000000000000000000000078FCE8
:42BAA800000000000000000000000000000000000000000000000000000000000000000000000000000000000000000000000000000000000000000000000000000000003CFE22
:42BAEA00000000000000000000000000000000000000000000000000000000000000000000000000000000000000000000000000000000000000000000000000000000003CFEE0
:42BB2C00000000000000000000000000000000000000000000000000000000000000000000000000000000000000000000000000000000000000000000000000000000003CFE9D
:42BB6E00000000000000000000000000000000000000000000000000000000000000000000000000000000000000000000000000000000000000000000000000000000003CFE5B
:42BBB000000000000000000000000000000000000000000000000000000000000000000000000000000000000000000000000000000000000000000000000000000000003CFE19
:42BBF200000000000000000000000000000000000000000000000000000000000000000000000000000000000000000000000000000000000000000000000000000000003CFED7
:42BC3400000000000000000000000000000000000000000000000000000000000000000000000000000000000000000000000000000000000000000000000000000000003CFE94
:42BC7600000000000000000000000000000000000000000000000000000000000000000000000000000000000000000000000000000000000000000000000000000000003CFE52
:42BCB800000000000000000000000000000000000000000000000000000000000000000000000000000000000000000000000000000000000000000000000000000000003CFE10
:42BCFA00000000000000000000000000000000000000000000000000000000000000000000000000000000000000000000000000000000000000000000000000000000003CFECE
:42BD3C00000000000000000000000000000000000000000000000000000000000000000000000000000000000000000000000000000000000000000000000000000000003CFE8B
:42BD7E00000000000000000000000000000000000000000000000000000000000000000000000000000000000000000000000000000000000000000000000000000000003CFE49
:42BDC000000000000000000000000000000000000000000000000000000000000000000000000000000000000000000000000000000000000000000000000000000000003CFE07
:42BE0200000000000000000000000000000000000000000000000000000000000000000000000000000000000000000000000000000000000000000000000000000000003CFEC4
:42BE4400000000000000000000000000000000000000000000000000000000000000000000000000000000000000000000000000000000000000000000000000000000003CFE82
:42BE8600000000000000000000000000000000000000000000000000000000000000000000000000000000000000000000000000000000000000000000000000000000002DFF4E
:42BEC8000000000000000000000000000000000000000000000000000000000000000000000000000000000000000000000000000000000000000000000000000000004078FE82
:42BF0A00000000000000000000000000000000000000000000000000000000000000000000000000000000000000000000000000000000000000000000000000000000003CFEBB
:42BF4C00000000000000000000000000000000000000000000000000000000000000000000000000000000000000000000000000000000000000000000000000000000003CFE79
:42BF8E00000000000000000000000000000000000000000000000000000000000000000000000000000000000000000000000000000000000000000000000000000000003CFE37
:42BFD000000000000000000000000000000000000000000000000000000000000000000000000000000000000000000000000000000000000000000000000000000000003CFEF5
:42C012000000000000000000000000000000000000000000000000000000000000000000000000000000000000000000000000000000000000000000000000000000008096FCDA
:42C0540008000000000000000000000000000000000000000000000000000000000000000000000000000000000000000000000000000000000000000000000000000000BCFEE8
:42C096000000000000000000000000000000000006008001000000000000000000000000000000000000000000000000000000000000000000000000000000000000000080FD64
:42C0D8000000000004401000000000000000000000000000000000000000000000000000000000000000000000008020000000000000000000000000000000000000000094FF9F
:42C11A00000000000020000000000000000000000000000000000000000000000000000000000000000000000000000100000000000000000000000000000000000000000CFDB9
:42C15C000000000004001000000000000000000000000000000000000000000000000000000000000000000000000020000000000000000000000000000000000000000018FF56
:42C19E00000000000000000000000000000000000000000000000000000000000000000000000000000000000000000000000000000000000000000000000000000000003CFE25
:42C1E0000200000000000000000000000000000000000000000000000000000000000000000000000000000000000000000000000000000000000000000000000000004058FE85
:42C2220008000000000000000000000000000000000000000000000000000000000000000000000000000000000000000000000000000000000000000000000000000000ADFF26
:42C26400000000000000000000000000000000000000000000000000000000000000000000000000000000000000000000000000000000000000000000000000000000003CFE5E
:42C2A600000000000000000000000000000000000000000000000000000000000000000000000000000000000000000000000000000000000000000000000000000000003CFE1C
:42C2E800000000000000000000000000000000000000000000000000000000000000000000000000000000000000000000000000000000000000000000000000000000003CFEDA
:42C32A00020000000000000000000000000000000000000000000000000000000000000000000000000000000000000000000000000000000000000000000000000000001CFEB5
:42C36C00000000000000000000000000000000000000000000000000000000000000000000000000000000000000000000000000000000000000000000000000000000003CFE55
:42C3AE0008000000000000000000000000000000000000000000000000000000000000000000000000000000000000000000000000000000000000000000000000000000BCFE8B
:42C3F000000000000000000000000000000000000000000000000000000000000000000000000000000000000000000000000000000000000000000000000000000000003CFED1
:42C43200000000000000000000000000000000000000000000000000000000000000000000000000000000000000000000000000000000000000000000000000000000003CFE8E
:42C47400000000000000000000000000000000000000000000000000000000000000000000000000000000000000000000000000000000000000000000000000000000003CFE4C
:42C4B6000000000020020048000900000440481080104002000008220024200400000000000000000000090041082004900012000002000100004800002001000000000048FC29
:42C4F80000000000A0000050000A404128002DA00000800050040A4001280005000000000000000050040A4001010105A00014900250000A00004001000005000000000078FE44
:42C53A0000000000200000400008000120000C800000000000000000000000000000000000000000000000000000000240000800012000040000800000000200000000006CFD50
:42C57C0000000000000000000000000000000000000000002000048000100002000000000000000020000480000000000000000000000000000000000000000000000000ECFE39
:42C5BE000017E002A8000950012A4005A8002DA0025C800B50012A4005A80015400200000000000950012A4005F80115A00254800A50012A800450011240054800092001E8FC60
:42C60000800C9001300506CA4019280365A04C9501324006CA4019280365A00C8001000000000006CA4019280364A20C9481325006CA40190003600A0C8029300006C00008FDD0
:02C64200FFFFF8
:00000001FF
